:020000040801F1
:1000000000000220BD1A01087D08010881080108CE
:1000100085080108890801088D0801080000000012
:10002000000000000000000000000000910801082E
:100030009508010800000000990801089D080108C2
:100040000D1B01080D1B01080D1B01080D1B0108EC
:100050000D1B01080D1B01080D1B01080D1B0108DC
:100060000D1B01080D1B01080D1B01080D1B0108CC
:100070000D1B01080D1B01080D1B01080D1B0108BC
:100080000D1B01080D1B01080D1B01080D1B0108AC
:100090000D1B01080D1B01080D1B01080D1B01089C
:1000A0000D1B01080D1B01080D1B01080D1B01088C
:1000B0000D1B01080D1B01080D1B01080D1B01087C
:1000C0000D1B01080D1B01080D1B01080D1B01086C
:1000D0000D1B0108AD080108B90801080D1B010836
:1000E0000D1B01080D1B01080D1B01080D1B01084C
:1000F0000D1B01080D1B01080D1B01080D1B01083C
:100100000D1B01080D1B01080D1B01080D1B01082B
:10011000C50801080D1B01080D1B01080D1B010876
:100120000D1B01080D1B01080D1B01080D1B01080B
:100130000D1B01080D1B01080D1B01080D1B0108FB
:100140000D1B01080D1B01080D1B01080D1B0108EB
:100150000D1B01080D1B01080D1B01080D1B0108DB
:100160000D1B01080D1B01080D1B01080D1B0108CB
:100170000D1B01080D1B01080D1B010800000000EC
:080180000D1B01080D1B010815
:10018800044B05481B1A062B02D9044B03B1184728
:10019800704700BF3300002030000020000000003E
:1001A80005490648091A891001EBD171491002D096
:1001B800034B03B11847704730000020300000207F
:1001C8000000000010B5064C237843B9FFF7D8FFAC
:1001D800044B13B10448AFF300800123237010BD12
:1001E8003000002000000000101B010808B5084B73
:1001F8001BB108490848AFF300800848036813B9E1
:10020800BDE80840CCE7064B002BF9D09847F7E744
:100218000000000034000020101B010830000020FE
:100228000000000070B50F4E0F4D761BB61018BFBA
:10023800002405D0013455F8043B9847A642F9D16B
:100248000A4E0B4D761B01F05FFCB61018BF002458
:1002580006D0013455F8043B9847A642F9D170BD41
:1002680070BD00BF381B0108381B01083C1B010882
:10027800381B010870B4860746D0541E002A41D0A6
:10028800CAB2034602E014F1FF343BD303F8012B52
:100298009D07F8D1032C2ED9CDB245EA05250F2CA0
:1002A80045EA054519D903F110022646103E0F2EDE
:1002B80042F8105C42F80C5C42F8085C42F8045CB6
:1002C80002F11002F2D8A4F1100222F00F0204F099
:1002D8000F041032032C13440DD91E462246043A4B
:1002E800032A46F8045BFAD8221F22F003020432DC
:1002F800134404F003042CB1C9B21C4403F8011BD5
:100308009C42FBD170BC704714460346C2E700BF4D
:10031800F0B595B008A830220021FFF7ABFF002404
:100328001D4A019404940394059406940794116C4F
:100338001A4B41F080511164126C02F08052019204
:10034800019A02941A6842F480421A601B680F945A
:1003580003F48043029301230225082148220B93CA
:1003680008A803231026109111921393029F089551
:100378000E9512950C9600F0ABFE0F224FF48053A9
:1003880003A829460495059407940392069301F05F
:1003980095F815B0F0BD00BF00380240007000406D
:1003A80010B5094C094920463223082200F098FC70
:1003B80020460B22064900F053FD42F21070BDE8BA
:1003C800104001F041BB00BF0401002000000020E4
:1003D80050000020444B454A454C80B59A6001F0D6
:1003E8000BFBFFF795FF00F0C9F800F09DF900F04E
:1003F80063F900F07DF90A2305223E493E4800F0E2
:100408006FFC4FF47A7001F01FFB0A2305223B4969
:10041800394800F065FC21464FF4FA631422364847
:1004280000F0BAFC0A2314222146354800F058FC93
:10043800A37C5A1E012A4FD9052B05D10A230B226A
:1004480030492F4800F04CFC2F4C304F304EDFF82D
:10045800CC80304DB3EE008AFFF7A2FFD4ED007ACE
:10046800F4EEC87AF1EE10FAF6D5384600224FF4C9
:10047800806101F021FA384600224FF4807101F0C2
:100488001BFA304600224FF4004101F015FA3046BD
:1004980000224FF4005101F00FFA304600224FF4C9
:1004A800006101F009FA404600224FF4004101F0D2
:1004B80003FA284600224FF4004101F0FDF92846CE
:1004C80000224FF4005101F0F7F900224FF40061C7
:1004D800284601F0F1F9BDE70A2307220E4908482A
:1004E80000F0FEFBB0E700BF00ED00E000000108EF
:1004F80070000020100000200401002008000020E7
:10050800C4000020200000204C0000200000024011
:10051800000C0240001002401800002000040240B5
:100528000268104B9A4200D070470F4B1A78012A84
:10053800FAD15A78032AF7D1F0B593F803E019797C
:100548005F799A79DE791B7A084D094C094801EBE5
:100558000E2102EB072203EB0623296022600360C9
:10056800F0BD00BF004400405000002060000020A3
:10057800640000205C000020704700BF2DE9F043B4
:100588008BB00024464B00941A6B464DDFF820913F
:10059800DFF82081444F454E42F001021A631A6B7E
:1005A80002F001020092009A01941A6B42F01002C4
:1005B8001A631A6B02F010020192019A02941A6BE4
:1005C80042F002021A631A6B02F002020292029AC5
:1005D80003941A6B42F008021A631A6B02F00802BD
:1005E8000392039A04941A6B42F004021A631B6B79
:1005F80003F004030493284601224FF47841049B36
:1006080001F05AF9484601224FF4404101F054F9EB
:10061800404601224FF47C4101F04EF93846012250
:100628004FF4007101F048F9012230464FF47C5133
:1006380001F042F9284605A901254FF478430593AE
:1006480007940894069501F021F8484605A94FF447
:100658004043059306950794089401F017F840461F
:1006680005A94FF47C43059306950794089401F077
:100678000DF8384605A94FF40073059306950794BD
:10068800089401F003F84FF47C5305A93046069509
:1006980007940894059300F0F9FF0BB0BDE8F083C8
:1006A80000380240001002400008024000000240EA
:1006B80000040240000C02400B4B0C4A10B50C2100
:1006C8001A604FF4E134002218465C6059619A6060
:1006D800DA601A619A61DA6100F0D2FA00B910BDE5
:1006E800BDE81040FFF748BFC4000020004C0040A0
:1006F8000B4B0C4A10B50C211A604FF4E134002260
:1007080018465C6059619A60DA601A619A61DA6128
:1007180000F0B6FA00B910BDBDE81040FFF72CBFD5
:1007280084000020001001400B4B0C4A10B50C212E
:100738001A604FF41644002218465C6059619A60AA
:10074800DA601A619A61DA6100F09AFA00B910BDAC
:10075800BDE81040FFF710BF04010020004400402E
:10076800F0B503683C4A934289B02BD03B4A934288
:100778004DD03B4A934201D009B0F0BD0024394B1B
:100788000294196C384841F4003119641B6C03F465
:10079800003302930322072303A9602702260125B9
:1007A800DDF808E00692079303970496059500F094
:1007B8006DFF22462146262001F0A6F8262001F0EA
:1007C800D9F8D9E70024274B0094196C274841F43D
:1007D800002119641B6C03F40023009303220823EF
:1007E80003A94FF4406702260125DDF800E00692D0
:1007F800079303970496059500F048FF2246214683
:10080800342001F081F8342001F0B4F8B4E7002472
:10081800144B0194596C164841F0100159645B6CF3
:1008280003F0100301930322072303A9C02702261C
:100838000125DDF804E006920793039704960595D1
:1008480000F024FF22462146252001F05DF82520EE
:1008580001F090F890E700BF004C00400010014004
:100868000044004000380240000C024000080240EA
:1008780000040240704700BFFEE700BFFEE700BF6C
:10088800FEE700BFFEE700BF704700BF704700BF2C
:10089800704700BF08B501F0C9F8BDE8084001F08D
:1008A80091B800BF014800F045BB00BF840000209C
:1008B800014800F03FBB00BF04010020014800F0E0
:1008C80039BB00BFC400002008B5032001F00AF8B6
:1008D800002211466FF00B0001F016F800221146B5
:1008E8006FF00A0001F010F8002211466FF00900BD
:1008F80001F00AF8002211466FF0040001F004F834
:10090800002211466FF0030000F0FEFF002211469E
:100918006FF0010000F0F8FF002211464FF0FF30A1
:10092800BDE8084000F0F0BF2DE9F04704682269EF
:100938008246C068DAF81C10DAF80830DAF8106075
:10094800DAF8145022F4405202432261E268DAF8DD
:100958001800334322F416422B4322F00C020B43B7
:100968001343E360636923F440730343B1F5004F15
:100978006361AB4B61D09C4200F0018103F5806359
:100988009C4200F0FC8000F051FEA64FDAF80430DB
:1009980000EB800000EB80009B00B0FBF3F3A7FBAB
:1009A80003235B091D0100F041FEDAF8043000EB77
:1009B80080009B0000EB8000B0FBF3F600F036FEF1
:1009C800DAF8042000EB8000930000EB8000B0FB15
:1009D800F3F3A7FB03234FF064095B0909FB1363D7
:1009E8001B013233A7FB03235B0903F0F00600F079
:1009F8001DFEDAF8042000EB8000930000EB800075
:100A0800B0FBF3F800F012FEDAF8043000EB8000D7
:100A18009B0000EB8000B0FBF3F0A7FB003040091F
:100A280009FB10831B013233A7FB0323C3F34313D2
:100A380033432B44A360BDE8F0879C425DD003F5A7
:100A480080639C4259D000F0F1FD764FDAF804300B
:100A580000EB800000EB80005B00B0FBF3F3A7FB2A
:100A680003235B091E0100F0E1FDDAF8043000EB16
:100A780080005B0000EB8000B0FBF3F500F0D6FDD2
:100A8800DAF8042000EB8000530000EB8000B0FB94
:100A9800F3F3A7FB03235B094FF0640909FB135326
:100AA800DB003233A7FB03231B0903F4F87500F0BE
:100AB800BDFDDAF8042000EB800000EB8000530055
:100AC800B0FBF3F800F0B2FDDAF8043000EB800078
:100AD80000EB80005B00B0FBF3F3A7FB03235B098B
:100AE80009FB1383DB003233A7FB0323C3F3421351
:100AF80033442B44A360BDE8F08700F0AFFD494FB5
:100B0800DAF8043000EB800000EB80005B00B0FBFB
:100B1800F3F3A7FB03235B091E0100F09FFDDAF83E
:100B2800043000EB80005B0000EB8000B0FBF3F5C5
:100B380000F094FDDAF8042000EB8000530000EB8D
:100B48008000B0FBF3F3A7FB03234FF064095B09B4
:100B580009FB1353DB003233A7FB03231B0903F400
:100B6800F87500F07BFDDAF8042000EB80005300F4
:100B780000EB8000B0FBF3F800F070FDA4E700F094
:100B88006DFD284FDAF8043000EB800000EB8000A0
:100B98009B00B0FBF3F3A7FB03235B091D0100F0E7
:100BA8005DFDDAF8043000EB80009B0000EB80006C
:100BB800B0FBF3F600F052FDDAF8042000EB8000F9
:100BC800930000EB8000B0FBF3F3A7FB03234FF087
:100BD80064095B0909FB13631B013233A7FB032379
:100BE8005B0903F0F00600F039FDDAF8042000EBA9
:100BF8008000930000EB8000B0FBF3F800F02EFDBE
:100C0800DAF8043000EB800000EB80009B00B0FBBA
:100C1800F3F3A7FB03235B0909FB138302E700BF78
:100C2800001001401F85EB512DE9F04107460E46A3
:100C380090461D463C6801E06B1C06D1206836EAE8
:100C48000003F9D10020BDE8F08135B100F0F6FECF
:100C5800A0EB08008542EDD23C68E36823F4D0732A
:100C6800E3606369202223F001030021636103200C
:100C780087F8392087F8381087F83A20BDE8F081DE
:100C880060B338B590F83930044603F0FF0203B377
:100C98002268242384F83930D36823F40053D360BE
:100CA8002046FFF741FE23681A6922F490421A6130
:100CB8005A6922F02A025A61DA680025202142F492
:100CC8000052DA602846E56384F8391084F83A104F
:100CD80038BD80F83820FFF743FDD9E70120704779
:100CE8002DE9F0430F4690F83910202983B003D03E
:100CF800022003B0BDE8F083002F3ED0002A3CD08C
:100D0800984690F83830012B0446F1D00020012194
:100D18002123E06384F8381084F83930019200F018
:100D28008DFE019AA2848146E28406E0FFF77CFFEB
:100D380028BB23683A785A600137E58CADB2434640
:100D48004A4680212046E5B1E58CA668013DADB252
:100D5800B6F5805FE584E9D143464A4680212046BE
:100D6800FFF762FF58B93B8821682269C3F308037B
:100D78004B60002AE0D10237DFE70120B9E7032002
:100D8800B7E74021FFF750FF0028F8D1202384F867
:100D9800380084F83930ACE72DE9F0430E4690F876
:100DA8003A10202983B003D0022003B0BDE8F083B5
:100DB80076B36AB3984690F83830012B0446F3D0DE
:100DC800002001212223E06384F8381084F83A30A7
:100DD800019200F033FE019AA2858146E285E58DF5
:100DE800ADB243464A462021204685B3E58DA76823
:100DF800013DADB2B7F5805FE58512D0FFF714FF6E
:100E080058BB236933B923685B6833700136E6E75A
:100E18000120CAE723685B6803F07F03337001365B
:100E2800DDE743464A4620212046FFF7FDFEA0B9EC
:100E3800236933B923685B68C3F3080326F8023BC8
:100E4800CDE723685B68DBB226F8013BC7E784F887
:100E58003850284684F83A10A7E70320A5E700BFD2
:100E680090F83A30202B01D002207047D9B1D2B186
:100E780090F83830012BF7D030B400230468C285CD
:100E88002225C36380F83A506569828545F00105DB
:100E9800816280F838306561E26842F490721846E1
:100EA800E26030BC70470120704700BF704700BF48
:100EB8008368B3F5805F28D0036973B10368826AD9
:100EC8005B68511C03F07F0381621370C38D013B83
:100ED8009BB2C38543B100207047836A0268591CDE
:100EE800526881621A70F1E70268D16821F4907142
:100EF80010B5D1605169202421F00101516180F8B9
:100F08003A40FFF70DFB002010BD0269836A3AB929
:100F180002685268C2F3080223F8022B8362D5E7FD
:100F280002685268D2B223F8012B8362CEE700BF71
:100F3800704700BF03681A6870B51607DD685969FD
:100F4800044649D011F0010152D0D60705D5E8056D
:100F580003D5E06B40F00100E06356077AD500291D
:100F680000F08480E16B900741F00201E16376D5DF
:100F7800E16B41F00401E163110772D4E16B0029D0
:100F880029D0910605D5AA0603D594F83A20222A35
:100F98007CD05D69E16B0E0702D415F040057AD06C
:100FA800DA6822F49072DA605A69202122F001028C
:100FB8005A6184F83A105A6955065ED55A69606BC9
:100FC80022F040025A61002857D03B4B036500F0DD
:100FD80077FC002855D170BD96060CD5A9060AD510
:100FE80090F83A30222BF6D1BDE87040FFF760BF89
:100FF80015F4907FA9D110060ED45606EBD56D06D0
:10100800E9D5DA68202122F04002DA60204684F827
:101018003910FFF74BFF70BD2906EED594F839203B
:10102800212AD8D1A268B2F5805F226A38D0511C33
:10103800216212785A60E28C013A92B2E284002A64
:10104800C9D1DA6822F08002DA60DA6842F0400238
:10105800DA6070BD96070BD5002989D18EE7110794
:101068008CD5E16B41F00801E16387E7900785D4EF
:10107800100783D5002981D0F3E72046FFF758FFF2
:1010880070BD606BBDE87040036D18472046FFF7E0
:101098000FFF23687DE72046FFF74AFFE56370BD31
:1010A80011882069C1F30801596010B9023222621F
:1010B800C1E701322262BEE7C510010808B5836B9B
:1010C8000022DA851846DA84FFF732FF08BD00BF30
:1010D800F0B50368DD0783B004462FD5A3498A68B5
:1010E80002F00C02042A00F0F4808A6802F00C0274
:1010F800082A00F0EA806368B3F5803F00F02C818D
:10110800B3F5A02F00F00081984D2A6822F48032B0
:101118002A602A6822F480222A60002B40F0FD8091
:1011280000F08CFC064605E000F088FC801B642873
:1011380000F2AA802B689B03F6D423689F072DD55D
:101148008A4A916811F00C0F00F0A580916801F0AF
:101158000C01082900F09B80E368002B00F0EB806D
:10116800834B824D01221A6000F068FC064605E0B8
:1011780000F064FC801B022800F286802B68980728
:10118800F6D52968F82292FAA2F22369B2FA82F215
:1011980021F0F80193400B432B6023681A0720D4F1
:1011A800590734D4A369CBB1704DAA6802F00C0278
:1011B800082A77D0022B6F4B4FF000021A6000F01C
:1011C800D18000F03BFC2C46054604E000F036FCDC
:1011D800401B022858D823689B01F7D4002003B08D
:1011E800F0BD6369002B60D0634B604D01221A602B
:1011F80000F024FC064604E000F020FC801B0228D6
:1012080042D86B6F9F07F7D523685907CAD5574B44
:101218005A4D002201921A6C42F080521A641B6CDB
:1012280003F080530193019B2B6843F480732B6078
:1012380000F004FC064604E000F000FC801B0228D5
:1012480022D82B68DA05F7D5A368012B00F0F180C6
:10125800052B00F0D580454D2A6F22F001022A6740
:101268002A6F22F004022A67002B40F0D28000F097
:10127800E5FB41F2883607462B6F980792D500F0B8
:10128800DDFBC01BB042F7D9032003B0F0BD5268A4
:1012980056023FF561AF354A1268950723D5E268D3
:1012A800012A20D0012003B0F0BD334A2F4D13602E
:1012B80000F0C4FB064604E000F0C0FB801B0228D7
:1012C800E2D86B6F9807F7D49EE74A6850027FF51B
:1012D80012AF264A126891037FF530AF6268002A80
:1012E8007FF42CAFDEE7214DF821286891FAA1F1AF
:1012F8002269B1FA81F120F0F8008A4002432A609D
:101308001A077FF54DAF6CE7184B1A6842F4802234
:101318001A601A6842F480321A6000F08FFB134D8D
:10132800064604E000F08AFB801B6428ACD82B68D2
:101338009A03F7D501E70E4A0C4D136000F07EFBC7
:10134800064604E000F07AFB801B02289CD82B6834
:101358009907F7D4236821E7044A136843F48033D4
:101368001360DAE700F06AFB06460FE00038024037
:101378000000474260004742800E4742007000402C
:1013880000F05CFB801B02283FF67EAF2B689901BA
:10139800F6D447F6C07696FAA6F64FF44032B6FA77
:1013A80086F692FAA2F24FF07061B2FA82F091FAE0
:1013B800A1F1A26A676AE369D4F820E0E46A5208F6
:1013C80043EA0E0307FA06F6013A8240B1FA81F1C0
:1013D800334304FA01F11343194A1A4C0B43012110
:1013E8006B60116000F02AFB054605E000F026FB63
:1013F800401B02283FF648AF23689A01F6D5EDE670
:10140800104B1A6F42F004021A671A6F42F0010279
:101418001A6700F013FB0B4D074641F288362B6F15
:101428009B073FF5BFAE00F009FBC01BB042F6D9E1
:101438002AE7044A136F43F001031367E9E700BF83
:101448006000474200380240194A936803F00C03D1
:10145800042B2BD0082B27D15168536801F03F018A
:1014680013F4800F536847F6C07292FAA2F0B0FAEC
:1014780080F003EA020323FA00F314BF0D480E4874
:10148800B0FBF1F000FB03F0094B4FF440325B680E
:1014980092FAA2F2B2FA82F203F44033D340013353
:1014A8005B00B0FBF3F07047034870470148704792
:1014B8000038024040787D010024F400574A136840
:1014C80003F00F038B4208D2CBB21370136803F0FA
:1014D8000F03994201D00120704703689A072DE94C
:1014E800F04106D54E4C8568A26822F0F0022A43E6
:1014F800A260DF0706460C4626D54268012A00F09E
:101508008780931E012B464B1B687BD9990728D5EA
:10151800434DAB6823F003031343AB6000F08EFA2E
:101528007368012B074641F288384FD0022B58D0F8
:10153800032B05D160E000F081FAC01B404564D858
:10154800AB6813F00C0FF6D1344A136803F00F039D
:101558009C4209D2E3B21370136803F00F039C4254
:1015680002D00120BDE8F08133685A0706D52C491E
:10157800F0688A6822F4E05202438A601B0707D5A4
:10158800274A3169936823F4604343EAC1039360AF
:10159800FFF75AFF224B0146F0229B6892FAA2F20B
:1015A800B2FA82F203F0F003D3401E481E4AC35C2D
:1015B800002021FA03F3136000F008FA0020BDE8C8
:1015C800F08100F03BFAC01B40451ED8AB6803F021
:1015D8000C03042BF5D1B7E700F030FAC01B4045E7
:1015E80013D8AB6803F00C03082BF5D1ACE700F077
:1015F80025FAC01B404508D8AB6803F00C030C2B38
:10160800F5D1A1E7980183D4ABE70320BDE8F081C9
:10161800034B1B689D033FF57BAFA2E7003C0240EC
:1016280000380240281B01082C000020084B4FF40A
:10163800E0529B6892FAA2F2B2FA82F203F4E05303
:10164800D3400449044ACB5C1068D840704700BFB7
:1016580000380240281B01082C000020084B4FF4DA
:1016680060429B6892FAA2F2B2FA82F203F46043F3
:10167800D3400449044ACB5C1068D840704700BF87
:1016880000380240281B01082C0000202DE9F04FEB
:10169800D1F800C0DFF81482DFF814E283B0002527
:1016A80003E00135102D00F09B800123AB4003EAD5
:1016B8000C029342F5D14E6826F0100ABAF1020FD7
:1016C80000F091804FEA45090324D0F800B004FAED
:1016D80009F4E44306F003070BEA040B07FA09F7D9
:1016E8000AF1FF3A47EA0B07BAF1010F076040F227
:1016F800A080C7688B683C4003FA09F32343C360A2
:10170800F300CED54FF00009CDF80490D8F8443056
:1017180043F48043C8F84430D8F8444025F0030324
:1017280003F1804304F4804403F59C33019405F0ED
:101738000304019FD3F808A0A4000F27A7402AEAB2
:10174800070A544FB84222D007F58067B84200F024
:101758008380514FB84200F08480504FB84200F067
:1017680085804F4FB84200F086804E4FB84200F057
:1017780087804D4FB84200F08880DFF8389148459F
:101788000CBF4FF007094FF0080909FA04F94AEAB3
:1017980009079F60DEF80030D443F70354BF2340A5
:1017A8001343CEF80030DEF80430B70354BF2340AB
:1017B8001343CEF80430DEF80830F70254BF234054
:1017C8001343CEF80830DEF80C30B60205F10105F7
:1017D80054BF23401343102DCEF80C307FF465AF6F
:1017E80003B0BDE8F08F4FEAD50900EB890905F091
:1017F8000707D9F82040BF004FF00F0B0BFA07FB83
:1018080024EA0B0A0C69BC4044EA0A04C9F82040DF
:101818004FEA45090324D0F800A004FA09F4E44388
:1018280006F003070AEA040A07FA09F747EA0A076B
:101838000760876807EA040ACF6807FA09F747EAE2
:101848000A078760D0F804A0C6F300172AEA030342
:10185800AF401F4347604CE74FF0010909FA04F90C
:1018680095E74FF0020909FA04F990E74FF00309E8
:1018780009FA04F98BE74FF0040909FA04F986E735
:101888004FF0050909FA04F981E74FF0060909FA4A
:1018980004F97CE70000024000080240000C024006
:1018A80000100240001402400018024000380240B4
:1018B800003C0140001C024002B9090481617047E4
:1018C80090F83530022B03D0802343650120704700
:1018D8000268052380F83530136823F0010313608C
:1018E80000207047074AD3684FF6FF010B400002FB
:1018F80043F0BF6300F4E06043F400330343D36074
:10190800704700BF00ED00E0184B70B4DC68C4F30A
:101918000224C4F10706042E04F1040328BF042698
:10192800062B17D9033C0125A540013D2A40012378
:10193800B340013B1940A140002841EA02010CDBF9
:1019480000F1604000F561400901C9B280F8001358
:1019580070BC704700221446E9E7054B00F00F0001
:1019680009010344C9B2197670BC704700ED00E064
:10197800FCEC00E000F01F0101234009024A8B4003
:1019880042F82030704700BF00E100E00138B0F1B4
:10199800807F0ED2084B10B4084C5860F02084F8B1
:1019A80023000022072110469A6019605DF8044B55
:1019B80070470120704700BF10E000E000ED00E034
:1019C800704700BF08B5FFF7FBFF08BD084B094A81
:1019D8001B6810B5A2FB032304469809FFF7D6FF3E
:1019E800214600224FF0FF30FFF78EFF002010BD88
:1019F8002C000020D34D621008B50B4B1A6842F436
:101A080000721A601A6842F480621A601A6842F416
:101A180080721A600320FFF765FF0020FFF7D6FFEA
:101A2800FEF752FF002008BD003C0240024A13683E
:101A380001331360704700BF44010020014B186850
:101A4800704700BF4401002010B582B00190FFF735
:101A5800F5FF0446FFF7F2FF019B001B9842F9D3FC
:101A680002B010BD1049114BD1F8882042F4700221
:101A780010B4C1F888201A680D4C002042F0010209
:101A88001A6098601A6822F0847222F480321A6010
:101A98005C601A684FF0006422F480221A60D860F3
:101AA8008C605DF8044B704700ED00E000380240A0
:101AB80010300024DFF834D0002103E00C4B5B58D1
:101AC800435004310B480C4B42189A42F6D30B4A48
:101AD80002E0002342F8043B094B9A42F9D3FFF78E
:101AE800C1FFFEF79FFBFEF775FC70470000022060
:101AF800401B0108000000203000002030000020BA
:101B080048010020FEE70000F8B500BFF8BC08BC9B
:101B18009E467047F8B500BFF8BC08BC9E467047A3
:101B2800000000000102030401020304060708097B
:041B3800F5010108AA
:041B3C00CD010108CE
:101B400001030000000305CBFE00010001000000BE
:101B5000FE00020002000000636F6E6E6563740099
:101B60006E6F7420636F6E6E656374000024F40002
:0400000508011ABD17
:00000001FF
